:020000040000FA
:040000006A303A2800
:08000800A000030EA100831209
:1000100005191028831601178312B23081002B288E
:1000200083160113831203140B190310A80DA90DD5
:10003000AA0DAB0DAC0DAC16FF302C02031D2B2806
:10004000FA302B02031D2B2831152A08AF0029088E
:10005000AE002808AD008B100B11210E8300A00EFE
:04006000200E090065
:0C007400203084008001840A6030040207
:10008000031C3C281230B00056228316FF23900038
:10009000831283160C308505870183128501870141
:1000A000073099000030831691008312C830831600
:1000B0008100831231309000003083168C0083124F
:1000C00010308B00831600309B001C141A0883121A
:1000D000BC00851D63233C1C7C28831610309B00CC
:1000E0001C141A088312BD00831630309B001C14A8
:1000F0001A088312C200ED22831620309B001C14C4
:100100001A088312C1000130C1080319C10081011E
:100110008E018F010B118B100B108C018B179F2000
:100120003119A2203522B30B9D2803108519031421
:10013000B90DF03039020319C42102238F2864005D
:100140003210080031110130B7008B13203037070F
:1001500083169B001C141A088312A4001030370762
:1001600083169B001C141A088312A300A6000230F9
:10017000A6060030370783169B001C141A0883124A
:10018000A200A7000130A7068B17321CCD28220938
:100190000339A200A309A409A50924082F02031DFD
:1001A000BE2923082E02031D472922082D02031D04
:1001B000BE2901303702031DE4283C19E3283D180D
:1001C000E4283D143E14572202303702031DEF2865
:1001D0003C19EE28BD18EF28BD143E145E220330F2
:1001E0003702031DFA283C19F9283D19FA283D1554
:1001F0003E14652204303702031D05293C190429E9
:10020000BD190529BD153E146C2205303702031DAA
:1002100010293C190F293D1A10293D163E1473224E
:1002200006303702031D1B293C191A29BD1A1B2948
:10023000BD163E147A2207303702031D26293C19C9
:1002400025293D1B26293D173E14812208303702FF
:10025000031D31293C193029BD1B3129BD173E141E
:10026000882209303702031D3C293C193B294218DA
:100270003C2942143E148F220A303702031D4729BD
:100280003C194629C2184729C2143E149622260852
:100290002E02031DBE2927082D02031DBE29013091
:1002A0003702031D5A293C1959293D1C5A293D1072
:1002B0003E149D2202303702031D65293C19642932
:1002C000BD1C6529BD103E14A12203303702031D59
:1002D00070293C196F293D1D70293D113E14A5223E
:1002E00004303702031D7B293C197A29BD1D7B2967
:1002F000BD113E14A92205303702031D86293C1981
:1003000085293D1E86293D123E14AD220630370256
:10031000031D91293C199029BD1E9129BD123E143F
:10032000B12207303702031D9C293C199B293D1F30
:100330009C293D133E14B52208303702031DA7291E
:100340003C19A629BD1FA729BD133E14B9220930A7
:100350003702031DB2293C19B129421CB2294210AF
:100360003E14BD220A303702031DBD293C19BC29A9
:10037000C21CBD29C2103E14C122BE29B70A0B30CF
:10038000370203180800A5280130B600B300B400F6
:10039000B500B70085018701B1139F20B30B042A74
:1003A000031085190314B90DF030390203192B2AF3
:1003B000B40B042A013037020319C5220230370278
:1003C0000319C922033037020319CD220430370242
:1003D0000319D122053037020319D522063037021E
:1003E0000319D922073037020319DD2208303702FA
:1003F0000319E122093037020319E5220A303702D6
:100400000319E9229630B400311DCD293111321C77
:100410000E2A2D090339AD00AE09AF092F1CCD29D5
:100420008E018F010C1CCD290C102E1ECD298B1393
:1004300020303707BB002F08BA004322103037079F
:10044000BB002E08BA00432200303707BB002D083E
:10045000BA0043228B1785018701B70AB6010B301A
:100460003702031CCD29ED2208003E1C08003E1077
:100470001030BB003D08BA0043223030BB004208B8
:10048000BA00432208008B133A0883161C159A0001
:100490003B089B0055309D00AA309D009C146400D1
:1004A0009C184F2A1C1183128B1708000800051690
:1004B00040084107D0000F08D10008008516400809
:1004C0004107D2000F08D300080005144008410777
:1004D000D4000F08D5000800851440084107D60055
:1004E0000F08D7000800871440084107D8000F08FC
:1004F000D9000800071540084107DA000F08DB00A3
:100500000800071440084107DC000F08DD00080060
:10051000871640084107DE000F08DF0008000716B5
:1005200040084107CC000F08CD000800871540089F
:100530004107CE000F08CF00080005128E018F0181
:10054000080085128E018F01080005108E018F01B1
:10055000080085108E018F01080087108E018F0121
:10056000080007118E018F01080007108E018F010E
:10057000080087128E018F01080007128E018F017B
:10058000080087118E018F0108000508103A8500C8
:1005900008000508203A850008000508013A850092
:1005A00008000508023A850008000708023A87009B
:1005B00008000708043A870008000708013A870086
:1005C00008000708203A870008000708103A87004B
:1005D00008000708083A870008003D180516BD18EE
:1005E00085163D190514BD1985143D1A8714BD1AC9
:1005F00007153D1B0714BD1B871642180716C218A6
:10060000871508003C1D080050084002031D0D2BF3
:1006100051080F02031C0D2B051252084002031D46
:10062000162B53080F02031C162B85125408400288
:10063000031D1F2B55080F02031C1F2B0510560806
:100640004002031D282B57080F02031C282B85107E
:1006500058084002031D312B59080F02031C312B8F
:1006600087105A084002031D3A2B5B080F02031C37
:100670003A2B07115C084002031D432B5D080F0253
:10068000031C432B07105E084002031D4C2B5F0820
:100690000F02031C4C2B87124C084002031D552BE4
:1006A0004D080F02031C552B07124E084002031D74
:1006B0005E2B4F080F02031C5E2B87110C1C0800D9
:1006C0000C10C00A0800B601B301B4013C1C6B2B2E
:1006D000BC01BC14722BBC1C702BBC013C15722BD2
:1006E000BC013C143C08B6006400762B772B782BB9
:1006F000792B7A2BB41B0516B41F0512B30B742B80
:10070000B40B742B0310B60CB608031D742B003009
:0A071000BB003C08BA0043220800B9
:084000000900030002000600A4
:02400E00CC01E3
:10420000010078007A007C007E007B0079007F004E
:104210007D007A0078007E007C00FF00FF00FF0038
:104220000000F200F600FA00FE00F200F600FA00CC
:10423000FE00F200F600FA00FE00FF00FF00FF00A3
:10424000010005000500050005000900090009003E
:1042500009000D000D000D000D00FF00FF00FF0024
:10426000FF00FF00FF00FF00FF00FF00FF00FF0056
:10427000FF00FF00FF00FF00FF00FF00FF00FF0046
:10428000FF00FF00FF00FF00FF00FF00FF00FF0036
:10429000FF00FF00FF00FF00FF00FF00FF00FF0026
:1042A000FF00FF00FF00FF00FF00FF00FF00FF0016
:1042B000FF00FF00FF00FF00FF00FF00FF00FF0006
:1042C000FF00FF00FF00FF00FF00FF00FF00FF00F6
:1042D000FF00FF00FF00FF00FF00FF00FF00FF00E6
:1042E000FF00FF00FF00FF00FF00FF00FF00FF00D6
:1042F000FF00FF00FF00FF00FF00FF00FF00DD00E8
:00000001FF
